:020000040800F2
:1000000030040020AF3A0008EF380008EF3800084D
:10001000EF380008EF380008EF3800080000000053
:100020000000000000000000000000001D39000872
:100030001D390008000000001D390008C7380008FD
:100040001D3900081D3900081D3900081D39000838
:100050001D3900081D390008453900086D390008B0
:1000600095390008BD390008E53900081D39000838
:100070001D3900081D3900081D3900081D39000808
:100080001D3900081D3900080B3A00081D39000809
:100090001D3900081D3900081D3900081D390008E8
:1000A0001D3900081D3900081D3900081D390008D8
:1000B000333A00085B3A0008833A00081D3900080B
:1000C0001D3900081D3900081D3900081D390008B8
:1000D0001D3900081D3900081D3900081D390008A8
:1000E0001D3900081D3900081D3900081D39000898
:1000F0001D3900081D3900081D3900081D39000888
:100100001D3900081D3900081D3900081D39000877
:100110001D3900081D3900081D3900081D39000867
:100120001D3900081D3900081D3900081D39000857
:100130001D3900081D3900081D3900081D39000847
:100140001D3900081D3900081D3900081D39000837
:100150001D3900081D3900081D3900081D39000827
:100160001D3900081D3900081D3900081D39000817
:100170001D3900081D3900081D3900081D39000807
:100180001D3900081D390008AE010008FFFF1F2DB2
:100190002D2D204D6563726973702D5374656C6CE1
:1001A0006172697320322E352E32202D2D2DC6011D
:1001B00000084200043264757000386847F8046D26
:1001C000043F38607047D80100086200053264724D
:1001D0006F70043740CF7047F601000844000532C5
:1001E0007377617007CF043F386047F8046D043FB0
:1001F0003A600E0070470A020008620004326E691D
:10020000700007CF043F38607047240200084400A4
:1002100005326F766572B86847F8046D043F386040
:10022000FE68704748020008440005327475636B2D
:1002300007CF043F386047F8046D043F3A60043F3D
:100240003960043F386070476A0200084600043293
:10025000726F74003868B9683A69B86039613A6099
:1002600079687E60FE68F96070478C02000846007D
:1002700005322D726F743868B9683A69386139602F
:10028000BA60F968FE607E6879607047A002000875
:10029000200003323E7201CF01B440B440CF70471A
:1002A000B802000820000332723E47F8046D40BCDB
:1002B00001BC043F38607047D002000820000332C0
:1002C000724047F8046D019E47F8046D009E704728
:1002D000E2020008200006327264726F700002B001
:1002E0007047FA02000842000364322F3868F107B1
:1002F000761040080843386070470E03000862001B
:100300000364322A38680018764138607047280341
:10031000000842000464736872003868F1077608C8
:1003200040080843386070473E03000862000464D8
:1003300073686C0038680018764138607047500365
:1003400000084200046461627300002E07D4704705
:100350006E030008420007646E6567617465386863
:100360000021C043F64301304E4138607047860398
:100370000008640002642D0007CF121AB1410E007C
:10038000043F3A6070479C030008640002642B003D
:1003900007CF12184E41043F3A607047AE03000881
:1003A000610003733E6447F8046DF6177047C2039B
:1003B0000008620003756D2A3868A0FB06063860E5
:1003C0007047D60300086200026D2A00386880FB7F
:1003D0000606386070471404000844000375642A58
:1003E00007CF564341437618010C130C5943761836
:1003F000010C80B292B25143434350430022C918CA
:1004000052411204B6180A04090C80184E41043FE8
:1004100038607047A604000844000475646D2A0023
:1004200010B5002447F8046D7E6847F8046D3E69F6
:10043000FFF7C2FF310040CF300040CF47F8046DD6
:100440003E6847F8046DFE6803B4FFF7B5FF03BCD0
:10045000330040CF320040CF47F8046D3E6847F884
:10046000046D3E690FB4FFF7A7FF0FBC92196341FB
:1004700040CF89196241634140CF47F8046D7E68DF
:1004800047F8046DFE680FB4FFF796FF0FBC921992
:10049000634140CF89196241634140CF1E003A60F9
:1004A0007960B86010BDC80400084300022A2F001C
:1004B00000B540B440CFFFF789FF47F8046D40BC5A
:1004C00000F04CF8043700BDEA0400084300052A98
:1004D0002F6D6F6400B540B440CFFFF777FF47F84A
:1004E000046D40BC00F03AF800BD0C050008430064
:1004F00003752A2F00B540B440CFFFF75DFF47F8E2
:10050000046D40BC00F01BF8043700BD3005000846
:10051000430006752A2F6D6F640000B540B440CFCC
:10052000FFF74AFF47F8046D40BC00F008F800BD33
:1005300050050008430006756D2F6D6F640000B50F
:1005400047F8046D002600F019F840CF043700BDCD
:100550006E0500084300056D2F6D6F6400B547F808
:10056000046DF61700F032F840CF043700BDC00527
:10057000000844000675642F6D6F640030B40023DA
:1005800000227968B86835003C684026400049413F
:1005900052415B41AB4202D804D3A24202D3121BA8
:1005A000AB410130013EF1D10E0038607B60BA6092
:1005B00030BC704730B400237A68B9680020E2E7A5
:1005C00036060008440005642F6D6F6400B5F0170F
:1005D00019D0FFF7C4FEFFF705FEF0170CD0FFF7A8
:1005E000BEFEFFF7FFFDFFF7C9FFFFF7FBFDFFF7BB
:1005F000B6FEFFF7F7FD00BDFFF7F4FDFFF7BEFF06
:10060000FFF7ADFE00BDFFF7EDFDF0170ED0FFF7D1
:10061000A6FEFFF7E7FDFFF7B1FFFFF7A0FEFFF72C
:10062000E1FDFFF79CFEFFF7DDFD00BDFFF7DAFD02
:10063000FFF7A4FF00BD4C060008440002642F0031
:1006400000B5FFF7C3FFFFF7DCFD00BD940600080F
:10065000440002662A0000B5F0170DD0FFF77FFEB8
:10066000FFF7C0FDF0170DD0FFF779FEFFF7D8FEBA
:1006700040CF01CF386000BDFFF7B4FDF017F5D0D3
:10068000FFF76DFEFFF7CCFE40CF01CF3860FFF7DC
:1006900066FE00BDE0060008440002662F0000B5BB
:1006A000F0170ED0FFF75BFEFFF79CFDF0170ED0A2
:1006B000FFF755FEFFF796FDFFF77CFFFFF7A1FD63
:1006C00000BDFFF78FFDF017F4D0FFF748FEFFF7EE
:1006D00089FDFFF76FFFFFF742FEFFF792FD00BDB8
:1006E000F406000820000232210006CF316072605B
:1006F00040CF704708070008200002324000043F46
:1007000070683860366870471C070008440003644E
:10071000753C07CF121AB141B64170473007000847
:1007200044000364753E07CF801A8E41B64170477E
:1007300046070008440002643C0007CF121AB1418A
:100740000CDB0026704762070008440002643E008C
:1007500007CF801A8E4101DB002670470026F64342
:1007600070477207000862000364303C0437F617D4
:1007700070478607000862000364303D01CF0643DE
:10078000013EB6417047A0070008440003643C3EA8
:1007900007CF50404E400643013EB641F6437047F6
:1007A000B8070008440002643D0007CF50404E40A7
:1007B0000643013EB6417047CA0700082000037394
:1007C000704047F8046D3E007047DA0700082000CB
:1007D00003737021370040CF7047EC0700082000FA
:1007E0000372704047F8046D6E467047FC070008BE
:1007F000200003727021B54640CF70470C080008F6
:1008000061000364757047F8046D70471C080008A8
:1008100061000464726F700040CF704732080008B6
:100820006100043F64757000002E01D047F8046D2C
:1008300070474608000862000473776170003968E9
:100840003E600E007047540800086200036E697035
:1008500004377047680800086200046F766572000C
:1008600047F8046D7E6870477E08000862000474D3
:1008700075636B0001CF083F7E6038607047940855
:100880000008630003726F7403CF083F78603E6016
:100890000E007047AC0800086300042D726F7400EE
:1008A00003CF083F7E60396006007047BE0800082D
:1008B0002000047069636B0057F826607047D60803
:1008C00000080000056465707468BC49C91B47F8DE
:1008D000046D8E107047F20800080000067264650F
:1008E0007074680047F8046D6E46B549891B8E1018
:1008F0007047020900082000023E720040B440CF59
:10090000704714090008200002723E0047F8046D89
:1009100040BC70472609000820000272400047F8DA
:10092000046D009E7047360900082000057264724D
:100930006F7001B070474A090008200005727069A5
:10094000636BB6006E4436687047600900086E003D
:1009500003616E6401CF064070470640000616F042
:10096000780900086E000362696301CFB043060096
:1009700070478643000636F08E0900086E00026F4D
:10098000720001CF064370470643000656F0A409E3
:1009900000086E0003786F7201CF464070474640F2
:1009A000000696F0B20900086100036E6F74F6430A
:1009B0007047C2090008610003636C7AB6FA86F6D4
:1009C0007047D009000861000373687276087047A9
:1009D000DE09000861000373686C76007047EE0959
:1009E0000008610003726F725FEA76067047000AC2
:1009F0000008610003726F6CB61956F1000670476B
:100A00001A0A00086C00067273686966740001CFE8
:100A1000F0400600704736080026340A00086C00D3
:100A2000076172736869667401CF304106007047D0
:100A30003610F6174E0A00086C00066C736869667B
:100A4000740001CFB04006007047360000265E0AF1
:100A50000008610002303D00013EB6417047700A57
:100A60000008610003303C3E013EB641F64370474A
:100A70007E0A0008610002303C00F6177047940AB5
:100A80000008600004747275650047F8046D002664
:100A9000F6437047A80A000860000566616C73653C
:100AA00047F8046D00267047BC0A00084200023E69
:100AB0003D0001CFB042EADA00267047D00A0008B4
:100AC0004200023C3D0001CFB042E0DD002670470D
:100AD000E20A00084200013C01CFB042D7DB002609
:100AE0007047F40A00084200013E01CFB042CEDC5C
:100AF00000267047080B0008620003753E3D01CFD9
:100B0000861BB641F64370471C0B00086200037554
:100B10003C3D01CF361AB641F64370472E0B000814
:100B2000620002753C0001CF861BB6417047400B46
:100B30000008620002753E0001CF361AB6417047C8
:100B4000560B00086B00023C3E0001CF361A013EF6
:100B5000B641F6437047680B00086B00013D01CFBA
:100B6000361A013EB64170477C0B00086200036DE7
:100B7000696E01CFB04200DC06007047900B0008A0
:100B80006200036D617801CFB04200DB0600704760
:100B9000A60B0008620004756D61780001CFB042B9
:100BA00000D306007047C40B0008620004756D692D
:100BB0006E0001CFB04200D806007047300300201D
:100BC00030040020020C00080000046D6F76650000
:100BD00007B5310040CF320040CF00290FD0B242DC
:100BE0000DD006D3013E013A705C50540139FBD15F
:100BF00005E030781070013601320139F9D140CF6B
:100C000007BD240C000800000466696C6C0030000D
:100C100040CF310040CF002902D001397054FCD1BF
:100C200040CF7047300C0008200001403668704704
:100C3000480C00086D00012103CF30600E007047A2
:100C400006607047016070476E0C00086D00022B53
:100C5000210003CF3268121832600E00704702681C
:100C600092190260704702685218026070477C0C4B
:100C7000000820000268400036887047960C000883
:100C80006D000268210003CF30800E00704706809F
:100C9000704701807047BC0C00086D0003682B2171
:100CA00003CF3288121832800E00704702889219E2
:100CB000028070470288521802807047CA0C0008F0
:100CC00020000263400036787047E40C00086D0095
:100CD0000263210003CF30700E007047067070472A
:100CE000017070470A0D00086D0003632B2103CFCC
:100CF0003278121832700E00704702789219027022
:100D000070470278521802707047320D00086D006B
:100D100004626973210003CF3268024332600E001F
:100D20007047026832430260704702680A430260FB
:100D300070475A0D00086D0004626963210003CFFB
:100D40003268824332600E0070470268B24302602C
:100D5000704702688A4302607047820D00086D0088
:100D600004786F72210003CF3268424032600E0077
:100D70007047026872400260704702684A40026031
:100D80007047EC0D0008680004626974400001CFF0
:100D90003668064018BF4FF0FF3670474FF4D04218
:100DA00000B5012B0AD147F8046D002600F0CAFFF8
:100DB00047F8046D160001F02FFB11E002CF013B54
:100DC00002F0BCFC47F8046D3626164301F024FB04
:100DD00047F8046D0E0047F8046D002600F0B2FFDE
:100DE00047F8046D8A4E01F0FFF800BD140E0008AC
:100DF0006D0005686269732103CF32880243328037
:100E00000E007047028832430280704702880A430E
:100E1000028070473C0E00086D000568626963211E
:100E200003CF3288824332800E0070470288B2437B
:100E30000280704702888A4302807047640E00086F
:100E40006D000568786F722103CF3288424032808E
:100E50000E007047028872400280704702884A4044
:100E600002807047840E000868000568626974405B
:100E700001CF3688064018BF4FF0FF3670474FF459
:100E800008428DE7AC0E00086D00056362697321AE
:100E900003CF3278024332700E007047027832433B
:100EA0000270704702780A4302707047D40E00083F
:100EB0006D0005636269632103CF3278824332702B
:100EC0000E0070470278B2430270704702788A437E
:100ED00002707047FC0E00086D000563786F722188
:100EE00003CF3278424032700E0070470278724071
:100EF0000270704702784A40027070471C0F000869
:100F0000680005636269744001CF3678064018BFF7
:100F10004FF0FF3670474FF4F04241E72C0F0008C6
:100F200061000563656C6C2B04367047640F000824
:100F300061000563656C6C73B600704700F0EAFCF5
:100F40001E466C6173682063616E6E6F742062650B
:100F5000207772697474656E2074776963650A001E
:100F600002F013BC4C1000080000083136666C61BA
:100F7000736821003FB54FF00F00304015D000F0EE
:100F8000C9FC223136666C61736821206E65656428
:100F9000732031362D616C69676E6564206164640D
:100FA000726573730A0002F0F0BB30680130C5D17E
:100FB00070680130C2D1B0680130BFD1F068013033
:100FC000BCD1144A144B1360144B1360144A4CF2F6
:100FD000FA331360134A144B136008CF04CF02CFC7
:100FE00001CF01C602C600F021F804C608C600F011
:100FF0001DF80C4A10684FF0010188431060094A3F
:1010000010684FF000410843106040CF3FBD000022
:10101000920D00080840005823016745AB89EFCDC9
:1010200010400058144000580100000107B4284A3D
:101030004FF4803110680842FCD14FF00101106874
:101040000842FCD08843106007BC7047EC100008D1
:1010500000000E666C61736870616765657261732C
:1010600065000FB5300040CF1A4B98422FD31A4A73
:101070001A4B13601A4B13604FF00C01C8404FF02D
:10108000FF0108404FF0030188404FF00201084380
:10109000144A10604FF48031084310600C4A136802
:1010A0004FF480301840FAD10E4A10684FF00041DA
:1010B000084310600C4A116802B44FF4C0608143C9
:1010C00011604FF4C0500143116002BC11600FBDAC
:1010D00010400058004000080840005823016745B0
:1010E000AB89EFCD14400058004000586A11000849
:1010F00000000A6572617365666C6173680022485E
:1011000072B622494FF6FF72038893421CD047F80B
:10111000046D060047F8046D00F0FCFB1045726199
:10112000736520626C6F636B20617420200000F097
:1011300059FC00F0EFFB0C2066726F6D20466C616D
:1011400073680A00FFF78DFF02308842DCD100F09F
:10115000E1FB1246696E69736865642E20526573FF
:10116000657420210A0002F09CFB90110008000029
:101170000E6572617365666C61736866726F6D008F
:10118000300040CFBCE700000040000800000C0821
:10119000B2110008000009696E6974666C617368B9
:1011A00053484FF420710022027001300139FBD105
:1011B00070479812000800000768666C6173682128
:1011C00030B5320040CF500813D300F0A3FB1E68A7
:1011D000666C61736821206E656564732065766551
:1011E0006E206164647265737365732E0A0002F089
:1011F000CCBA404B9A4210D200F08CFB1943616E7E
:101200006E6F7420777269746520696E746F2063E5
:101210006F726520210A02F0B8BA13093448202100
:10122000046824099C4226D014300139F8D1304892
:1012300020210468002C17D014300139F9D100F0B6
:1012400069FB21546F6F206D616E79207363617447
:10125000746572656420466C617368207772697486
:1012600065732E0A02F091BA1B01036001394160D7
:101270008160C16001610F2111400431465240CFAD
:101280000168013101600F221140082903D100F0EB
:101290001AF8FFF76FFE30BDF812000800000A666A
:1012A0006C757368666C6173680000B51048202126
:1012B0000268002A03D000F006F8FFF75BFE143046
:1012C0000139F5D100BD47F8046D466847F8046D53
:1012D000866847F8046DC66847F8046D066947F8E4
:1012E000046D0F26F6430268164000220260704724
:1012F00030040020004000080E1300086900012B94
:1013000001CF3618704736180036000616F1241340
:1013100000086900012D01CF861B7047361A003E78
:101320000006B6F132130008610002312D00013EC3
:10133000704740130008610002312B0001367047EE
:101340004E130008610002322D00023E70475C130C
:101350000008610002322B00023670476E1300084D
:101360006100066E656761746500764270478013A0
:101370000008610003616273F01736184640704739
:101380009E130008420005752F6D6F6401CF310078
:10139000B0FBF6F67143401A043F38607047BC1347
:1013A00000084200042F6D6F640001CF310090FBF4
:1013B000F6F67143401A043F38607047D0130008B6
:1013C0004200036D6F6400B5FFF7EFFF40CF00BD33
:1013D000E01300086200012F01CF90FBF6F6704782
:1013E000F01300086A00012A01CF464370474643C4
:1013F000FE130008610002322A00760070470C14C8
:101400000008610002322F00761070472014000897
:101410006100046576656E00012030403618704723
:1014200038140008810004626173650047F8046D98
:10143000894E70470A0000004E1400080000066242
:10144000696E6172790084480221016070476414FA
:101450000008000007646563696D616C7E480A21BD
:1014600001607047B81400080000036865787A4886
:1014700010210160704779494FF0FF0008607849FA
:101480004FF48040086077494AF2050008607649C9
:101490004FF00100086075494FF0EE400860744954
:1014A0004FF02300086073494FF480500860724980
:1014B0004FF00D0008607047D414000881000968DF
:1014C0006F6F6B2D656D697447F8046D6B4E7047D7
:1014D000BE150008F0140008810008686F6F6B2DBE
:1014E0006B65790047F8046D654E7047E415000898
:1014F0000E15000881000A686F6F6B2D656D6974A9
:101500003F0047F8046D5F4E70470E1600082A151D
:101510000008810009686F6F6B2D6B65793F47F894
:10152000046D594E70473C160008481500088100AC
:101530000A686F6F6B2D70617573650047F8046DF5
:10154000524E7047523800085E15000800000465CE
:101550006D6974000FB5494800F026F80FBD72158B
:1015600000080000036B65790FB5454800F01CF8D2
:101570000FBD84150008000005656D69743F414882
:1015800000688746961500080000046B65793F00E7
:101590003D4800688746AC1500080000057061757D
:1015A00073653A480068874600688746D215000888
:1015B00000000B73657269616C2D656D697400B50F
:1015C00000F025F8002E40CFFAD0314A167040CFF7
:1015D00000BDFA15000800000A73657269616C2D80
:1015E0006B65790000B500F029F8002E40CFFAD0E5
:1015F00047F8046D274A167800BD2A160008000037
:101600000C73657269616C2D656D69743F0000B57E
:10161000FFF7C7FF47F8046D00261F4801684FF029
:101620008000014000D0F64300BD9C160008000079
:101630000B73657269616C2D6B65793F00B5FFF7BF
:10164000B0FF47F8046D0026134801684FF02000F2
:10165000014000D0F64300BDFCFF01204C000058C3
:1016600060000058000400481804004820040048A6
:101670000C3801400838014000380140F8FF0120D3
:10168000F4FF0120F0FF0120ECFF0120E8FF012022
:1016900028380140243801401C380140C016000899
:1016A0000000076365787065637400B5386801B43D
:1016B0000130386000F00BF801BC067040CF00BD6F
:1016C000361700080000066163636570740000B59A
:1016D00002CF01390022FFF747FF300040CF7F28BB
:1016E00009D0202819D2092816D00A281FD00D2881
:1016F0001DD00828EFD1002AEDD000F00BF9030827
:101700002008002AE7D0885C013A80230340E2D019
:1017100040230340F5D0DEE72020B242DBD247F879
:10172000046D0600FFF716FF01328854D3E7160058
:1017300000F09FF800BD481700084000037469627C
:1017400047F8046D294E70475E1700088100033E7C
:10175000696E47F8046D264E70470000000084173C
:10176000000882000E63757272656E742D736F755A
:101770007263650047F8046D1E4E7047000000005C
:1017800068000020A0170008000009736574736FDB
:1017900075726365174802CF0660416040CF70479D
:1017A000BE170008000006736F757263650047F886
:1017B000046D104E043F7068386036687047F81743
:1017C000000800000571756572790FB508480021A1
:1017D0000160FFF7B5FF47F8046D47F8046DC826B0
:1017E000FFF775FFFFF7D6FF0FBD00006800002070
:1017F000E4FF0120DCFF012040180008000007631F
:101800006F6D706172650FB5310040CF01CF8842B6
:1018100002CF10D1002810D001380A5C335C412A75
:1018200002D35B2A38BF2032412B02D35B2B38BF57
:1018300020339A42EED000260FBD0026F6430FBD9E
:101840005418000800000263720000B500F062F84E
:10185000010A00BD66180008000002626C0047F82B
:10186000046D202670477A18000800000573706127
:10187000636547F8046D20266CE69A18000800009E
:10188000067370616365730000B5002E03DDFFF71A
:10189000F0FF013EFBD140CF00BDAA180008500068
:1018A000065B636861725D0005E0C2180008000015
:1018B00004636861720000B501F0DBFB40CF36784D
:1018C00000BDD21800085000012847F8046D2926F1
:1018D00006E0EC1800085000015C47F8046D002693
:1018E00000B501F0D0FB043740CF00BD301900082F
:1018F0003000022E2200AA4800B547F8046D060009
:1019000000F07DFA47F8046D222601F0BCFB00F0E0
:10191000BDFD00BD0AB447F8046D7646013E33783C
:101920000121013319405B181EEB030E0ABC39E09C
:10193000561900083000026322009A48DCE747F895
:10194000046D7646013E33780121013319405B185E
:101950001EEB030E7047801900083000027322004E
:101960009148C9E747F8046D764647F8046D013E93
:1019700036780121731C19405B181EEB030E70476B
:1019800098190008000005636F756E74013647F8FA
:10199000046D013E36787047B019000800000563F9
:1019A0007479706500B5FFF7F1FF00F007F800BD2E
:1019B000D8190008000004747970650001B501CFE2
:1019C000002E07D047F8046D0678FFF7C3FD0130FD
:1019D000013EF7D140CF01BD121A00080000046893
:1019E00065782E0007B5310040CF20200F22043843
:1019F00047F8046D0E00C6401640092E01D937364F
:101A000000E03036FFF7A6FD0028F0D1FFF731FFE8
:101A100007BD221A0008000003682E731FB5634C2F
:101A20000EE0321A0008000003752E731FB5604CDB
:101A300006E0D61A00080000022E73001FB55D4CA8
:101A40005D49C91B8908220A2020292F200A202845
:101A5000273E200A202F43432020203335204343B4
:101A6000430A385C29295F200A0A544A106803B4E3
:101A70000A201060FFF74EFF08537461636B3A2031
:101A80005B0047F8046D0E0001F0D5FCFFF742FF44
:101A9000025D200003BC2736484A106000290AD0A6
:101AA000474A106806B447F8046D0600A04706BC14
:101AB000043A0139F5D1FFF72DFF0620544F533A70
:101AC000200047F8046D3600A047FFF723FF0420ED
:101AD0002A3E0A001FBD761B0008000005776F72C2
:101AE000647300B5FFF716FF010A00F036FFFFF739
:101AF00011FF09416464726573733A2047F8046DFD
:101B0000FFF770FFFFF706FF064C696E6B3A200087
:101B100047F8046D3668FFF765FFFFF7FBFE0746E1
:101B20006C6167733A2047F8046DB688FFF75AFF77
:101B3000FFF7F0FE06436F64653A2000B01D00F029
:101B400048FF47F8046D0600FFF74CFFFFF7E2FE81
:101B5000064E616D653A200047F8046D0636FFF7C2
:101B600021FFFFF7D7FE010A00F010FF300040CF41
:101B7000BDD040CF00BDC81B0008000006756E75C3
:101B80007365640000B500F0D4FF4FF000500168A9
:101B90004FF00052914200D20A4E761A00BD00006A
:101BA000141900083E19000864190008E519000816
:101BB000273400083734000830030020FCFF0120E0
:101BC0002C03002000000C082C1D000800000D3123
:101BD00032626974656E636F64696E670FB5FF2E5C
:101BE00004D847F8046D5FF0FF360FBD16F0FF1004
:101BF000B0420ED14FF6FF710840310C814208D13E
:101C000016F0FF0656F4805647F8046D5FF0FF3675
:101C10000FBD16F0FF20B0420FD14FF6FF71084004
:101C2000310C814209D1360A16F0FF0656F40056EF
:101C300047F8046D5FF0FF360FBDFF223100114001
:101C4000300A1040884210D1300C104088420CD12C
:101C5000300E1040884208D116F0FF0656F4405668
:101C600047F8046D5FF0FF360FBD300000210131F1
:101C7000001850F100007FF07F020240802A05D05A
:101C80001F29F4D347F8046D00260FBD0829F9D3A6
:101C9000060036F0800611F00100C001064311F085
:101CA0000E00C002064311F010008005064347F8FD
:101CB000046D5FF0FF360FBD47F8046DDFF89C66DA
:101CC0005FF4704110EA0102120116435FF40061F3
:101CD00010EA0102D20316435FF4E06110EA010248
:101CE00012011643FF2110EA010216431E43BDE311
:101CF00047F8046DDFF868665FF0704110EA010292
:101D0000120B16435FF0006110EA010252081643FD
:101D10005FF0E06110EA0102120B16435FF47F01ED
:101D200010EA0102120C16431E439FE3921D0008A5
:101D300000001072656769737465726C697465720E
:101D4000616C2C000FB5330040CF1B02FF2E05D86D
:101D500056F400561E4300F05FFB0FBDFFF73EFF39
:101D6000002E40CF06D0DFF8FC0506431E4300F0EE
:101D70007DFB0FBDF643FFF731FF002E40CF06D0AD
:101D8000DFF8E40506431E4300F070FB0FBDF64389
:101D90000BE0F21D00080000096D6F76776D6F761D
:101DA000742C0FB5330040CF1B02300040CFFFF73B
:101DB00083FF4FF6FF7110EA014001D0FFF798FF53
:101DC0000FBD0FB50136300040CF0023FFF774FF81
:101DD000FFF78EFF06E00FB5013647F8046D0026C9
:101DE000FFF7B0FF47F8046D44F2807600F014FB73
:101DF0000FBD581E000800000563616C6C2C0FB508
:101E0000330000F086FE300040CF1B1A043BDFF8A1
:101E10005C151940002906D0DFF85425914202D004
:101E2000BDE80F40D7E740CF5B08DFF8480540F238
:101E3000FF7119400843DB0A40F2FF3119400904E1
:101E400008439B0A13F001018906084347F8046D13
:101E5000060000F00BFB0FBD8E1E00080000086C92
:101E600069746572616C2C0008B547F8046D4FF613
:101E7000470600F0D1FA47F8046D46F6045600F024
:101E8000CBFA47F8046D0626FFF75CFF08BDB21ECB
:101E900000080000066372656174650000B500F01B
:101EA0003DF841F6CF60804747F8046DBEF101066A
:101EB00000BD0E1F0008200005646F65733E41F6EB
:101EC000CF60804747F8046DBEF10106704747F8C0
:101ED000046DBEF101064FF000521368DFF898144C
:101EE00009684FF00050834205D20F2008400428B3
:101EF00005D00231F9E70220084000D0023102315A
:101F00001160FFF75EFF136000F0D1F900BD781F8C
:101F100000080000073C6275696C647300B500F04E
:101F20009DFB4FF0005001684FF0005291420CD2DF
:101F300000F0EFFD0F200640042E40CF10D047F8F0
:101F4000046D362600F068FAF2E700F0E2FD0220A8
:101F5000064040CF04D047F8046D362600F05CFA06
:101F600047F8046D4BF2005600F056FA47F8046D3E
:101F70000A2600F0BEFA00BD841F00085000035B73
:101F8000275D03E09C1F00080000012700B501F059
:101F900070F800F05EFD300040CF00BDDA1F000891
:101FA000300008706F7374706F6E650000B5FFF7D6
:101FB000EDFF102101400DD12021014005D0FFF798
:101FC00053FF47F8046DED4E04E0FFF74DFF47F86F
:101FD000046DEB4EFFF713FF00BD3020000800003A
:101FE00007696E6C696E652C00B54BF200514BF6BB
:101FF000005244F270733088884208D0904208D072
:10200000984206D047F8046D060000F005FA023643
:10201000F1E740CF00BD0EB44BF6005244F27073AE
:1020200001880230914201D09942F9D10EBC70472B
:10203000462000080000047265742C0047F8046D07
:102040004BF60056E8E1542000083000046578693A
:102050007400F3E76C200008300007726563757246
:10206000736547F8046DC44E3668C8E684200008DE
:10207000810005737461746547F8046DC14E704743
:1020800000000000962000080000015DBD4800210E
:10209000C94301607047A62000081000015BB948E1
:1020A000002101607047CE2000080000013A00B511
:1020B000B548076000F0D2FA47F8046D4BF20056BD
:1020C00000F0AAF9AF480021C943016000BD2221F8
:1020D00000083000013B00B5AB480168B94214D09C
:1020E000AA498E4202D1AA4EFFF75CFCFFF712FC10
:1020F0001520537461636B206E6F742062616C6194
:102100006E6365642E0A01F040BB47F8046D4BF620
:10211000005600F081F900F0CAF89A4800210160E9
:1021200000BD362100080000076578656375746599
:10213000300040CF87464E210008100009696D6DC0
:1021400065646961746547F8046D1026E8E06421F0
:102150000008500006696E6C696E650047F8046DF2
:102160002026DDE07E21000810000B636F6D706992
:102170006C656F6E6C7947F8046D3026D0E098215D
:10218000000850000A302D666F6C6461626C650057
:1021900047F8046D4026C3E0B221000850000A3120
:1021A0002D666F6C6461626C650047F8046D4126B2
:1021B000B6E0CC21000850000A322D666F6C6461D5
:1021C000626C650047F8046D4226A9E0E62100082C
:1021D00050000A332D666F6C6461626C650047F8CD
:1021E000046D43269CE00022000850000A342D664E
:1021F0006F6C6461626C650047F8046D44268FE083
:102200001A22000850000A352D666F6C6461626CFA
:10221000650047F8046D452682E03422000850002E
:102220000A362D666F6C6461626C650047F8046D58
:10223000462675E04E22000850000A372D666F6C66
:102240006461626C650047F8046D472668E07E2291
:102250000008000008636F6E7374616E740000B54F
:1022600000F0FCF9FFF700FE47F8046D44F27076C9
:1022700000F0D2F8FFF78CFF00F019F800BDA022A3
:10228000000800000932636F6E7374616E7400B5EC
:1022900000F0E4F939683E600E46FFF7E5FDE1E73E
:1022A00010230008000006736D756467650000B5B3
:1022B0004FF0005001684FF00052914221D2023994
:1022C0000A884FF6FF739A4205D147F8046D4FF024
:1022D000000600F0A1F800F075F800F089F82D482C
:1022E000006847F8046D06002B49096804314FF077
:1022F00000521368116000F08FF81360FEF7D5FFED
:1023000000BD00F05FF847F8046D4FF0000608E0EC
:102310009C230008000008736574666C6167730095
:1023200000B54FF0005001684FF00052914205D2C5
:10233000184801683143016040CF00BD320040CFF2
:1023400015480068043001884FF6FF73994201D1A7
:10235000110000E01143018000BD0000000040F2C8
:102360000000C0F200005FF000007FF00100C0FF3D
:102370000000C0FF00F800F014000020E81F000873
:10238000FE1D0008D8FF012010000020851912044E
:10239000461A00082000002004000020B82300088E
:1023A000410007616C69676E656401203040361832
:1023B0000220304036187047E02300080000056115
:1023C0006C69676E00B54FF0005001680220014053
:1023D00005D047F8046D4FF0000600F01DF800BD71
:1023E0000E240008000008616C69676E31362C000D
:1023F00000B54FF0005001680F20014006D047F8AB
:10240000046D4FF0000600F007F8F2E700BD482425
:102410000008000002682C000FB5B6B24FF0005063
:1024200001684FF00052914205D247F8046D0E004A
:10243000FEF7C6FE02E0320040CF0A8047F8046D86
:10244000022600F056F80FBD622400080000012C9F
:1024500000B547F8046DFFF7DFFF360CFFF7DCFF30
:1024600000BD7E2400080000033E3C2C00B547F868
:10247000046D360CFFF7D0FFFFF7CEFF00BDE6245A
:102480000008000007737472696E672C07B5FF219E
:10249000314040CF300040CF002905D147F8046DCE
:1024A0000026FFF7B9FF07BD47F8046D067836022E
:1024B0000E43FFF7B1FF0130013902290AD347F873
:1024C000046D4678360202781643FFF7A5FF023006
:1024D0000239F2E7002900D107BD47F8046D0678FC
:1024E000FFF79AFF07BD44250008000005616C6CEA
:1024F0006F744FF0005001684FF0005291420FD2BC
:10250000320040CF89184A4A914219D3FFF702FAA4
:102510000B466C6173682066756C6C0A01F035B906
:10252000320040CF8918434A1268914208D3FFF71E
:10253000F1F90952616D2066756C6C0A01F025B9DC
:10254000016070476A250008000009666F726765C0
:102550007472616D00B500F028F84FF000503649F4
:10256000016036483649016000BD9625000800002C
:102570000D636F6D70696C65746F72616D3F47F8C4
:10258000046D00264FF0005000684FF00051884263
:102590004DD3F6437047BA25000800000C636F6DF9
:1025A00070696C65746F72616D004FF00050006867
:1025B0004FF00051884213D370474C2600080000AA
:1025C0000E636F6D70696C65746F666C6173680023
:1025D0004FF0005000684FF00051884200D2704721
:1025E0001648184902680B680A6003604FF00050F3
:1025F000154902680B680A6003600E480068834250
:1026000015D300B5FFF786F9232056617269616220
:102610006C657320636F6C6C69646520776974689E
:102620002064696374696F6E6172790A00BD7047D6
:1026300000000C0824000020D40600200400002024
:10264000880100081C000020180000205627000800
:1026500000000828637265617465290000B500F008
:1026600008FD002E0ED1FFF755F915204372656164
:102670007465206E65656473206E616D6520210A46
:1026800001F083B8386847F8046D043F386000F003
:10269000AFF940CF002E40CF11D0386847F8046D15
:1026A000043F3860FFF736F9095265646566696E64
:1026B0006520FFF783F9FFF72DF9022E2000FFF7C1
:1026C00081FE4FF0005000684FF00051884228D240
:1026D00095484FF000010160FFF78AFE47F8046D4E
:1026E0000C26FFF706FF00F014FA47F8046D0626E3
:1026F000FFF7FFFEFEF7D4F8FFF7C8FE8B4801682E
:102700000A684FF0FF339A4208D14FF00052136825
:10271000116047F8046DFFF79BFE1360066040CF21
:1027200013E000F0F6F9814847F8046D0668FFF7FA
:102730008FFE47F8046D4FF6FF76FFF76DFE7B487E
:10274000310040CF0160FFF7A1FE4FF0005001685B
:102750007748016000BD6E270008000008766172AE
:102760006961626C650047F8046D012613E08627F5
:102770000008000009327661726961626C6547F891
:10278000046D022607E0642800080000096E7661E7
:10279000726961626C6500B5FFF760FF4FF0005031
:1027A00001684FF00052914234D20F200640B2002F
:1027B00060480168891A604A91420BD2FFF7AAF873
:1027C0000F4E6F7420656E6F7567682052414D0A19
:1027D00000F0DBBF016047F8046D0E00FFF744FB1B
:1027E00047F8046D44F27076FFF716FE300040CFD4
:1027F0000200002805D00E600431FFF729FE0138E1
:10280000F9D147F8046D80261643FFF789FDFFF7DD
:102810004EFD00BD00F07DF90220064040CF04D1FE
:1028200047F8046D3626FFF7F7FD47F8046D434E71
:10283000FFF71CFE47F8046D414EFFF717FE47F8FF
:10284000046D44F27076FFF7E7FD300040CF0028BA
:1028500003D0FFF7FDFD0138FBD1FFF799FCFFF72F
:1028600026FD00BD44290008000007627566666504
:10287000723A00B5FFF7F2FE012030403618022010
:10288000304036184FF0005001684FF0005291422E
:1028900028D228480168891B274A91420BD2FFF7AA
:1028A00039F80F4E6F7420656E6F7567682052415E
:1028B0004D0A00F06ABF016047F8046D0E00FFF793
:1028C000D3FA47F8046D44F27076FFF7A5FDFFF7E1
:1028D000BFFD47F8046D40F24016FFF721FDFFF7FA
:1028E000E6FC00BD00F015F90220064040CF04D1FF
:1028F00047F8046D3626FFF78FFD47F8046D0F4E3D
:10290000FFF7B4FD47F8046D0D4EFFF7AFFD47F834
:10291000046D44F27076FFF77FFDFFF7EAFDFFF7E5
:1029200037FCFFF7C4FC00BD20000020040000209D
:102930001400002024000020D40600203E60043F44
:1029400002367E467629000800000F6469637469C8
:102950006F6E61727973746172744FF00050006829
:102960004FF0005147F8046D884201D2EA4E70479B
:10297000EA4E36687047B229000800000E646963A9
:1029800074696F6E6172796E6578740003B5316831
:102990004FF0FF30814207D08879FF2804D00E0025
:1029A00047F8046D002603BD47F8046D0026F64382
:1029B00003BDE429000800000A736B697073747228
:1029C000696E67003178013101220A408918761852
:1029D000704706B40178013101220A408918401875
:1029E00006BC70476C2A000800000466696E64002B
:1029F00030B500220023350040CF340040CFFFF730
:102A0000ACFF4FF6FF70B188884218D047F8046DCC
:102A10000636FEF7BBFF47F8046D260047F8046D45
:102A20002E00FEF7F0FE002E40CF08D0B01DFFF7BD
:102A3000D0FF02000B004FF00050824204D2FFF79B
:102A4000A5FF300040CFDCD0160047F8046D1E0013
:102A500030BD00B53100386803B4FFF7C9FF03BCCF
:102A60003A68002A01D100F05BFD00BDCC2A0008C5
:102A7000000006636A756D702C00320040CF310093
:102A800040CF8B1B043B6FF0FE01194000290ED094
:102A90006FF0FF0081420AD0FEF73CFF0D4A756DD2
:102AA0007020746F6F206661720A00F06EBE5B105A
:102AB000FF210B40134330001E0000B54FF00052C1
:102AC00013681060FFF7A8FC136000BD062B000818
:102AD0000000056A756D702C310040CF300040CF8A
:102AE0000B1A043B8E491940002902D08D4A9142AD
:102AF000D2D15B1040F2FF72134053F4604347F8A9
:102B0000046D1E00D9E71E2B0008000004686572E2
:102B1000650047F8046D4FF00056366870471A2C70
:102B2000000800000D666C6173687661722D68653F
:102B3000726547F8046D7C4E3668704700B547F8FB
:102B4000046D42F60066FFF767FC47F8046D4CF62B
:102B50004076FFF761FC00BDDBE700B500F03AF816
:102B600039683E600E4647F8046D4DF20016FFF7D7
:102B700084FF00BD00B500F02DF839683E600E46B8
:102B800047F8046D4DF20076FFF777FF00BD00B502
:102B9000FFF7D4FF00F01EF839683E600E4647F894
:102BA000046D4DF20006FFF768FF00BD00B500F0B0
:102BB00011F839683E600E46FFF78EFF00BD00B584
:102BC000FFF7BCFFFFF7A5FF47F8046D0226FFF7EC
:102BD00090FC00BD00B5FFF79CFF47F8046D02268E
:102BE000FFF787FC00BD00B5FFF793FFFFF774FF09
:102BF00000BD00B5FFF78DFF47F8046D4DF20006EC
:102C0000FFF73BFF00BD00B5FFF783FF47F8046DFA
:102C10004DF20016FFF731FF00BD562C00083000C2
:102C2000047468656E00052E01D140CFDBE7022EEB
:102C300001D140CFDDE7FEF76DFE17537472756367
:102C4000747572657320646F6E2774206D61746390
:102C5000680A00F09ABD722C0008300004656C739D
:102C6000650000B500F017F8FDF7BCFAFFF7DBFFD1
:102C700000BD8A2C000830000269660000B5FFF72D
:102C80009EFF47F8046D022600BDA42C000830000A
:102C900005616865616400B5FFF79CFF47F8046D46
:102CA000052600BDBE2C0008300006726570656107
:102CB000740000B500F01FF8FFF7B5FF00BDD62C7B
:102CC00000083000057768696C6500B5FFF7D6FF2E
:102CD000FDF788FA00BDEA2C0008300005756E7417
:102CE000696C012EA7D140CF51E7FE2C00083000BF
:102CF00005616761696E012E9DD140CF56E72C2D8D
:102D00000008300005626567696E00B5FFF724FFB3
:102D100047F8046D012600BD88010008040000206A
:102D200001F8FFFF00F8FFFF240000203C2D000801
:102D30002000016B47F8046D029E70474C2D00087F
:102D40002000016A47F8046D009E70475C2D000862
:102D50002000016947F8046D260070479A2D00088D
:102D60003000056C6561766500B5D84801683B00A8
:102D7000043F1A68043B1A6008338B42F9D103B44C
:102D8000FFF728FF03BC330040CF04390B6001601C
:102D900004390A6801320A6000BDAC2D0008200029
:102DA00006756E6C6F6F700030BC7047E42D0008C4
:102DB0003000052B6C6F6F70032E00D03BE740CFC7
:102DC00000B547F8046DC24EFFF70EF9FFF7D2FECB
:102DD0001AE014F10044641BA41940CF2C44A4F160
:102DE00000447047262E00083000046C6F6F70009E
:102DF000032E00D01FE740CF00B547F8046DB54E55
:102E0000FFF7F2F8FFF7A9FE00F019F9AF4831001B
:102E100040CF016047F8046DAF4EFFF7E5F800BD05
:102E20000134AC4270476E2E0008780002646F00D7
:102E300000B547F8046DA94EFFF7D6F8A34801681E
:102E400047F8046D0E0047F8046D00260760FFF791
:102E500083FE47F8046D032600BD00B500F02FF88F
:102E6000ECE730B4340040CF350040CF7047082F36
:102E700000087800033F646F00B547F8046D974E73
:102E8000FFF7B2F847F8046D44F2AC26FFF7C4FA36
:102E90008E48016847F8046D0E00FFF79BFE01366F
:102EA00047F8046D012689480760FFF755FE47F88B
:102EB000046D032600BD00B500F001F8E2E700B59F
:102EC00047F8046D4BF23046FFF7A6FA47F8046D59
:102ED0000426FEF737FF013B08D047F8046D0526AE
:102EE000FEF730FF013B00F029FC00BD47F8046D00
:102EF0003526FFF791FA47F8046D4CF64076FFF758
:102F00008BFA00F01BFC00BD222F00083000046388
:102F10006173650047F8046D002647F8046D0826C4
:102F20007047382F00083000033F6F666C4809E097
:102F3000013EB64140CF7047DE2F00087800026F97
:102F400066006848082E00D075E640CF00B547F807
:102F5000046D0600FFF748F8FFF73CFE39683E6055
:102F60000E46013647F8046D092647F8046D4CF605
:102F70004076FFF751FA00BD00B5300040CF013B6D
:102F800001B400F0DBFB01BC082E00D053E640CFBB
:102F900047F8046D0600FF213140B14205D14FF4DE
:102FA00038510E43FFF738FAD6E7FEF717FE002E2A
:102FB00040CF04D04C480643FFF758FACCE747F817
:102FC000046D0026FEF7BEFE47F8046D44F2B026FD
:102FD000FFF722FAC0E7300040CFB042704714300C
:102FE0000008300005656E646F66092E00D022E689
:102FF00040CF00B540B440CFFFF7ECFD39683E60EC
:103000000E46FFF700FE47F8046D40BC47F8046D1C
:10301000082600BD66300008300007656E646361F5
:103020007365082E00D006E640CF00B547F8046D62
:103030004CF64076FFF7F0F900F001F800BD00B55E
:10304000300040CF00280DD003B4012131400029C9
:1030500003D0013EFFF7CDFD01E0FFF7C4FD03BC47
:103060000138EFE700BD7A300008000005746F6B8F
:10307000656E47F8046D202605E0F4300008000076
:1030800005706172736510B5184801684068184A88
:1030900012688418202E07D191420FD0835CB3426E
:1030A00002D101328418F7E7914207D0835C0132E4
:1030B000B342F9D18618361B013E01E08618361B53
:1030C000043F3C600A48026010BD00000C00002074
:1030D000D22D0008202E0008A82D0008622E00081E
:1030E000302F0008D62F0008000FB6F1DCFF0120BA
:1030F000E4FF01203231000800000564696769744B
:10310000CF4B1B68303E0BD30A2E0BD3073E0A2E43
:1031100006D3242E06D3203E0A2E01D3242E01D31B
:10312000002670479E42FBD247F8046D0026F64306
:1031300070473C3200080000066E756D62657200D3
:103140003FB5310040CF701E0126012204B4BC4BB4
:103150001B680024002500293CD001300139027889
:103160002D2A04D101B00022D24304B4F3E7232A6C
:1031700001D10A23EFE7242A01D11023EBE7252A06
:1031800001D10223E7E72E2A01D10226E3E72C2A08
:1031900036D047F8046D1600FFF7B4FF002E40CF7D
:1031A0002BD047F8046D260047F8046D2E0047F831
:1031B000046D1E0047F8046D00260FB4FDF710F9EA
:1031C0000FBC350040CF340040CF0022A419554138
:1031D00040CFC0E704BC002A04D50022E443ED43FD
:1031E0000134554133002600012B02D047F8046D0D
:1031F0002E0047F8046D1E003FBD01B000263FBD04
:103200002500002402260029E4D0425C01392E2A40
:10321000F9D047F8046D1600FFF774FF002E40CF79
:10322000EBD0043F3C6047F8046D1E000FB4FDF77F
:1032300086F90FBC340040CF40CFE4E75E3200088F
:103240000000062E6469676974000A2E01D23036C8
:103250007047242E01D237367047232670479432A8
:103260000008000004686F6C6400330040CF7548AC
:1032700001783F290DD2013101704018012907D092
:103280000138027801300270013801390129F7D183
:1032900003707047B4320008000005686F6C643C2E
:1032A000330040CF674801783F2902D201310170D5
:1032B00043547047CC3200080000047369676E0005
:1032C000002E01D440CF70472D26CEE7E032000813
:1032D000000002233E005B480678013038607047EA
:1032E000F832000800000366235310B5202400F0D4
:1032F00008F8013CFBD110BD1A330008000002663B
:10330000230000B547F8046D4D4E3668FDF754F8BC
:10331000FFF79BFFFFF7C4FF00BD36330008000036
:103320000223530000B500F00AF8002EFBD13868E4
:103330000028F8D100BD623300080000012300B569
:1033400047F8046D3E4E366847F8046D0026FDF7D9
:1033500015F9FCF747FF40CFFFF777FFFFF785FF31
:1033600000BD743300080000023C230035480021F2
:103370000170704786330008000002662E0047F88F
:10338000046D202604E0D4330008000003662E6E8E
:1033900000B510B4340040CFFDF76CFAFCF7D5FF50
:1033A00047F8046D0026FFF7E1FFFFF7BBFF40CFB2
:1033B0002C26FFF775FF002C03D0FFF7A2FF013C7E
:1033C000FBD110BC40CFFFF77BFF47F8046D47F8F7
:1033D000046D1CE0EA33000800000375642E00B59C
:1033E000FFF7C4FFFFF79EFF11E01C340008000048
:1033F00002642E0000B5FDF73DFAFCF7A6FFFFF7CB
:10340000B5FFFFF78FFFFDF73FFAFFF759FFFFF713
:1034100062FFFEF7D3FAFEF72CFA00BD2E34000847
:10342000000002752E0047F8046D0026D7E74834E7
:1034300000080000012E47F8046DF617DAE70000D7
:10344000FCFF0120280000209034000800000865DF
:1034500076616C756174650000B5FEF7A8F901CF5F
:1034600001B440B440CFD948016802B400210160E2
:10347000FEF790F900F014F8D44802BC016047F858
:10348000046D40BC01BC043F3860FEF783F900BD09
:1034900062370008000009696E74657270726574A5
:1034A00030B5CB4887420BD9FEF734FA105374611C
:1034B000636B20756E646572666C6F770A0064E1F9
:1034C000C44887420AD2FEF725FA0F537461636B32
:1034D000206F766572666C6F770A56E1BE4C256880
:1034E000002D01D13D002560FFF7C3FD002E02D164
:1034F000043740CF30BD386847F8046D043F38606A
:10350000FFF776FA310040CF320040CF002A19D1C0
:1035100038683100FFF714FE320040CF002AC0D1D6
:1035200047F8046D060047F8046D0E00FEF746FAF2
:10353000FEF7F0F90C206E6F7420666F756E642EC6
:103540000A0022E1A54B1B68002B1DD10025256038
:1035500030230B40302B0ED1FEF730FAFEF7DAF9AC
:103560001220697320636F6D70696C652D6F6E6CCE
:10357000792E0A0009E1043740CF47F8046D1600A0
:10358000FEF7D6FDFFF78DFF043740CF80200840BF
:103590000ED1EB1B9B08402008400FD008200840AC
:1035A00002D0002B00D01DE00F200840834205D33D
:1035B00047F8046D1600FEF7BBFD72E700F0BEF899
:1035C00047F8046D160010220A4002D0FEF7B0FD45
:1035D00067E720220A4002D0FEF706FD61E7FEF70A
:1035E0000EFC5EE7072001401000FEF714FD0129E4
:1035F0001FD1012BDCD1FF213140B14204D14088E1
:103600000643FEF709FF4CE7FEF7E8FA002E40CF2D
:1036100004D040680643FEF729FF42E747F8046DEF
:103620000026FEF78FFB47F8046D0688FEF7F4FED0
:1036300037E7022902D1012BBAD1EFE7032927D1BD
:10364000012BB5D1FF213140B1420BD14FF478515C
:103650000E43FEF7E1FE043247F8046D1600FEF754
:10366000C3FC1EE7FEF7BAFA002E40CF04D05C4937
:103670000E43FEF7FBFEEEE747F8046D0026FEF76B
:1036800061FB023247F8046D1600FEF7ADFC08E757
:10369000042918D1012B8BD1330040CF002B00D14E
:1036A000FFE61F221A409A4205D047F8046D46886B
:1036B000FEF7B2FEF5E647F8046D06889B011E434F
:1036C000FEF7AAFEEDE6052924D1012B10D147F81B
:1036D000046D0026FEF736FB47F8046D0600FEF782
:1036E00083FC47F8046D4CF64076FEF795FED8E66D
:1036F00047F8046D0026FEF725FB47F8046D012608
:10370000FEF720FBFEF787FC47F8046D0600FEF786
:103710006BFCC6E606290ED1012B7FF449AFFEF7FC
:103720005DFA002E40CF3FF479AFD0F80200064397
:10373000FEF79CFEB5E601308047B2E600B5002BEF
:103740000CD0013B47F8046D1E0057F82660FEF7C9
:103750008BFB002BF5D1043D2F0040CF00252560C9
:1037600000BD7E370008810009686F6F6B2D717591
:10377000697447F8046D1B4E7047B6370008F83778
:1037800000080000047175697400DFF85CD0104F08
:10379000FDF706FD15480A2101601048002101606F
:1037A0000D480160094801601148016011494160FC
:1037B0000C4800688746FEF708F8FFF771FEFEF731
:1037C000A9F805206F6B2E0AF5E70000E4FF012041
:1037D000300300203001002008000020D8FF012025
:1037E0000006B6F1D4FF012030040020FCFF0120C8
:1037F000DCFF012068000020123800080000056589
:10380000696E743F47F8046DEFF31086013EB641D0
:1038100070472238000820000465696E740062B6A3
:1038200070473238000820000464696E740072B674
:10383000704748380008200004697073720047F828
:10384000046DEFF305867047543800080000036EDE
:103850006F70704796380008000009756E68616ED9
:10386000646C656400B5FEF755F814556E68616EBA
:10387000646C656420496E746572727570742000A2
:1038800047F8046DEFF30586FEF7ACF8FEF742F853
:1038900002210A0000BDA838000800000572657307
:1038A0006574C748C7490160D238000881000B69B8
:1038B00072712D7379737469636B47F8046DC24E2E
:1038C0007047643800084FF6D070C2F201000068FB
:1038D0008746FA3800088100096972712D666175A2
:1038E0006C7447F8046DB94E7047643800084FF6A1
:1038F000CC70C2F2010000688746283900088100B8
:103900000E6972712D636F6C6C656374696F6E0004
:1039100047F8046DAE4E7047643800084FF6C87023
:10392000C2F2010000688746503900088100096929
:1039300072712D657874693047F8046DA54E704733
:10394000643800084FF6C470C2F201000068874670
:10395000783900088100096972712D6578746931C0
:1039600047F8046D9C4E7047643800084FF6C070ED
:10397000C2F2010000688746A03900088100096989
:1039800072712D657874693247F8046D934E7047F3
:10399000643800084FF6BC70C2F201000068874628
:1039A000C83900088100096972712D65787469331E
:1039B00047F8046D8A4E7047643800084FF6B870B7
:1039C000C2F2010000688746F039000881000969E9
:1039D00072712D657874693447F8046D814E7047B3
:1039E000643800084FF6B470C2F2010000688746E0
:1039F000163A00088100076972712D61646347F807
:103A0000046D794E7047643800084FF6B070C2F20A
:103A10000100006887463E3A00088100086972711B
:103A20002D74696D320047F8046D704E704764382C
:103A300000084FF6AC70C2F2010000688746663A93
:103A400000088100086972712D74696D330047F8B0
:103A5000046D674E7047643800084FF6A870C2F2D4
:103A60000100006887468E3A00088100086972717B
:103A70002D74696D340047F8046D5E4E70476438EC
:103A800000084FF6A470C2F20100006887460C409F
:103A90000008FFFF182D2D2D20466C61736820440F
:103AA000696374696F6E617279202D2D2D00FDF7A9
:103AB000E2FC51488546514F2A264FF000505049AC
:103AC000016050485049016047F8046D4E4E4F4D1B
:103AD000B1884FF6FF73994225D04FF480730B40A5
:103AE0000AD0B01DFEF775FFFEF795FA03884088EF
:103AF00000040343ED1A16E080230B4013D00F237C
:103B0000194089006D1AB01DFEF763FFFEF783FAB6
:103B100047F8046D060047F8046D2E0047F8046D61
:103B20000E00FDF755F8FEF731FF300040CFCFD043
:103B30003748066040CF37480560374837494FF669
:103B4000FF72884204D0023803889342F9D00230D1
:103B500033490860FDF724FBFDF7DCFE384D656353
:103B6000726973702D5374656C6C61726973203265
:103B70002E352E3220666F722053544D3332574209
:103B80003535206279204D61747468696173204B0A
:103B90006F6368200A0023480021016047F8046D24
:103BA000214E47F8046D0426FEF722FF40CF002E79
:103BB00002D0FEF7BDFAFBE540CFE6E5696E697419
:103BC0000CED00E00400FA05D0FF0120CCFF01203D
:103BD000C8FF0120C4FF0120C0FF0120BCFF01205D
:103BE000B8FF0120B4FF0120B0FF0120ACFF01208D
:103BF000A8FF0120A4FF0120300400203003002092
:103C0000D4060020040000208801000800000220E3
:103C10001C0000202400002000000C0800400008C8
:0C3C20001800002008000020BC3B000839
:0400000508000000EF
:00000001FF
